:10000000C428A0007F39201B803C0920A01B003C95
:1000100008008A01820700340334063409340C34A2
:1000200010341334163419341C341F34223425345C
:1000300028342B342E3431343334363439343C3490
:100040003F3441344434473449344C344E345134D1
:100050005334553458345A345C345E34603462342A
:100060006434663468346A346B346D346F3470349D
:1000700071347334743475347634783479347A3432
:100080007A347B347C347D347D347E347E347E34EB
:100090007F347F347F347F34A4002508A402031CFE
:1000A000A5032708A602031CA7033709A2003509E8
:1000B000A300A20A0319A30A4130A900AC01AD01B3
:1000C000AE01AF01A801360884003409A7208413CB
:1000D000C0202408AC070318AD0A2508AD07260880
:1000E000AE070318AF0A2708AF072D080120803E8E
:1000F000A1002F080120803EA107210CA8070008BD
:100100003404031C34068000290303194130A9007C
:100110000319A20A0319A30F6828BF28003803197E
:10012000BF28A8002008840021188317A001A1017E
:10013000A81BA2280008A000A81CBF28840A000849
:10014000A100BF28AA200005031DA00ABF2884170C
:100150008005BF2800308A0028080739820701344B
:100160000234043408341034203440348034031012
:10017000A00DA10DFF3E0318B7282008BF28831348
:10018000031383126400080007309F006400051AFF
:10019000CA28C628003085190130BA000310BA0DEC
:1001A0000519BA0A0310BA0D8619BA0A0310BA0D56
:1001B0000619BA0A0310BA0D8618BA0A0310BA0D46
:1001C0000618BA0A1430BA023A08A2002A3C031CE4
:1001D00082290310220DA207F920A000A20AF9200B
:1001E000A100A20AF9208E202008B8002108B90039
:0A01F000822901308A00220800294C
:100200008207E73401340034C93401340034BA348D
:1002100001340034AB34013400349C3401340034F4
:100220008E340134003481340134003474340134A8
:1002300000346734013400344F3401340034E33483
:1002400004340034B93404340034903404340034B9
:100250006834043400344234043400341D3404342B
:100260000034F93403340034C43403340034A33488
:1002700003340034833403340034653403340034ED
:100280004734033400342B34033400340F34033444
:100290000034F53402340034DB3402340034C23428
:1002A00002340034AA34023400349334023400346B
:1002B0007C34023400346734023400345234023463
:1002C00000343E34023400342A340234003418340A
:1002D00002340034053402340034F4340134003480
:1002E000DA3401340034BA34013400349C3401343B
:1002F00000348134013400346734013400344F3425
:10030000013400340530B6000230B400B701B50145
:0E0310003908A700A5003808A6004C20822955
:02400E00CD3FA4
:00000001FF
